:0300000002234395
:0C234300787FE4F6D8FD75817702238ACC
:1028C5003F065B4F666D7D077F6F0008040C020AAB
:0A28D500060E0109050D030B070FA5
:102452006028800930304750524D432C30303030A4
:1024620030302C562C2C2C2C2C2C2C303030303064
:10247200302C2C2C412A30300A0000004180FA3CDA
:10293D00EF75F00A84FEEF75F00A84EEC454F0FED4
:03294D0025F0FF73
:012950002264
:10275A00E4FBFD7FD0122531E4FF12272CE4F53E7D
:10276A007412253EF582E43481F583E0FF12272CAA
:0C277A00053EE53EC3940740E71228DF4F
:012786002230
:0C298A009080E3E0FDE4FFFE1228F9223B
:0A29A100AD077F107E001228F92216
:0A29AB00AD077F207E001228F922FC
:1028A800EFC4540F9028CF93FEEF540F93FF7D048D
:0C28B8007804088002C333D8FCFF2EFF18
:0128C40022F1
:10282600300F07EFC4540FFC8004EF540FFC301038
:102836000AEC9028C593FF1228A822EC9028C5938D
:01284600FF92
:01284700226E
:10284800AB07E4FD7F9012253140107FAC12272C96
:102858007F0912272C1228DF7F00221228DF7F0130
:01286800224D
:102787008F3EAB3EE4FD7F9012253140177FEE125E
:10279700272C1228DF7423253EF582E43481F58344
:0A27A700E4F0FF221228DF7F012278
:1020C600AF8DEFFEAD8B7C00E42DF53FEC3EF53E8B
:1020D600908100E0FEA3E0FFE4FDFBFA7901F8122F
:1020E60019E4A804A905AA06AB07AE3EAF3FE4FC77
:1020F600FD1219D7E41217698F718E708D6F8C6E71
:102106007B007A247974784912165F8F718E708DF0
:102116006F8C6E7B007A40791C784612165F8F7141
:102126008E708D6F8C6EE4FFFEFDFCAB71AA70A9FC
:102136006FA86E1216FC6046AB71AA70A96FA86EE6
:10214600E4FFFE7D807C3F12165F1217A79080F891
:10215600EEF0A3EFF09080F8E0FAA3E0FB7C007DC0
:1021660064FFAE021218B49080FFEFF07C007D642D
:0F217600AF03AE021218B4908102EDF0C322D372
:012185002237
:1024D400300758C2073009289080E97444F0A37487
:1024E40020F0E4A3F0A3F0A37408F0A3EFF0A37426
:1024F400FFF0A3F0A3F0E4A3F0A3F0753E0B80106B
:102504009080E97402F0A37423F0A3EFF0753E0306
:102514007B017A8079E9A209920FC210AD3E1223A1
:0C252400CF5004D207C322D207D322C339
:012530002288
:102602001228DF9080E2E0FF2401F582E43480F5B5
:1026120083E004F074012FF582E43480F583E0D383
:102622009404401E9080E2E0FF2423F582E434818A
:10263200F5837401F074312FF582E43480F58374EC
:0326420001F02282
:10002600122579121FFE920BD207D20CD20DC214E2
:10003600C2057572017573817574087575017576DB
:10004600817577057F207E001229288F24E524D329
:10005600940840089080E87408F080069080E8E5EF
:1000660024F0E49080E2F09080E8E0FF9080E2E007
:10007600C39F5035E0FF2423F582E43481F5837471
:1000860001F01228489080E2E0FE2431F582E43443
:1000960080F583EFF074012EF582E43480F583EF6A
:1000A600F09080E2E004F080BE7811E62402F524A8
:0700B600E52478116670F9E2
:1000BD00D293300211C202908104E0600914F0E085
:1000CD007004C2A8D207300506A2B292968005A28E
:1000DD00B2B39296904000E044C0F5389080FEE0B7
:1000ED006538600DAF381224D450069080FEE53887
:1000FD00F09080FAE0FF7811E6C39F5003020241B1
:10010D00E4F69080E2E0FF9408502A74232FF582E4
:10011D00E43481F583E0701D9080E2E02423F582C4
:10012D00E43481F5837401F074312FF582E4348069
:10013D00F5837401F09080E2E004F09080E8E0FF38
:10014D009080E2E0C39F4008E4F09080FEE0F4F080
:10015D009080E2E0FF2431F582E43480F583E060A5
:10016D00211228489080E2E0FE2431F582E43480AB
:10017D00F583EFF074012EF582E43480F583EFF012
:10018D0080589080E2E0FF2401F582E43480F5830D
:10019D00E0B4020D74312FF582E43480F5837401DF
:1001AD00F09080E2E0FF122787BF01129080E2E01D
:1001BD002401F582E43480F583E004F0801C908006
:1001CD00E2E0FF2423F582E43481F583E4F0740149
:1001DD002FF582E43480F583E4F0C28EC2AAE49058
:1001ED008100F0A3F0F58DF58B9081037464F0C25E
:1001FD00037811E62402F538C20875B80C7811E6BB
:10020D00FFB53804D208800330B3F2EF2402F5387D
:10021D00E5387811667004D208800320B3F2200807
:10022D000AD28ED2ABC28BD2AA8009E49080FFF0A5
:10023D00908102F0E4FBFD7FD012253150030204C2
:10024D006CE4FF12272C1228DFE4FB7D017FD01216
:10025D0025315003020467C20F1226FA908112EF66
:10026D00F0547F6006200C0302041F753801C20F85
:10027D001226FA74122538F582E43481F583EFF0F5
:10028D002014090538E538C3940F40E2D20F122629
:10029D00FA1228DF300D167F107E001229288F24C8
:1002AD00E52430E004C2098002D209C20D9081120A
:1002BD00E030E71D20141AE4FBFD7FD0122531E458
:1002CD00FF12272C908112E0547FFF12272C122849
:1002DD00DF30140302044B300C1EC20CE4FFFE127F
:1002ED0029289080E3EFF07E007C0E7D101218A27D
:1002FD00908110EEF0A3EFF0908114E0FF54F0F533
:10030D002BC4540FF52B75F00AA4F52BEF540F25C4
:10031D002BF52B908116E0FF54F0F528C4540FF502
:10032D002875F00AA4F528EF540F2528F528A3E029
:10033D00FF54F0F527C4540FF52775F00AA4F527DF
:10034D00EF540F2527F527A3E0FF54F0F53AC454D9
:10035D000FF53A75F00AA4F53AEF540F253AF53A30
:10036D0024D0F526E43407F525908113E0FF54F0F1
:10037D00F52AC4540FF52A75F00AA4F52AEF540F87
:10038D00252AF52AE4F529F52C752D00752E25F570
:10039D002F753000753129852F41853042853143C8
:1003AD00AB2CAA2DA92E1222B68F358E348D338CFF
:1003BD00322093089081217401F08005E490812111
:1003CD00F0AF35AE34AD33AC32852F458530468533
:1003DD003147908121E0F548AB2CAA2DA92E121C96
:1003ED0040AF2B12293D9080D5EFF0AF2812293D5B
:1003FD009080D7EFF0AF2712293DA3EFF0E526242B
:10040D0030FF12293DA3EFF0908113E09080D4F0DE
:10041D00802CD20F1226FA1228DF908112E030E7DD
:10042D001D20141AE4FBFD7FD0122531E4FF1227A5
:10043D002C908112E0547FFF12272C1228DF90811F
:10044D0012E0547FFF908000E06F6016D20AE490B6
:10045D00810FF0908000EFF080081228DF800312EA
:10046D0028DF9080E2E0FB2423F582E43481F583DC
:06047D00E06003020660CE
:10048300FD7F90122531500302065D7FAC12272CAD
:10049300920E9080E2E0FB7D017F901225315003A4
:1004A30002065D7F0A122996D20F1226FA8F245371
:1004B3002480E52470030206589080E2E0FBE4FD0B
:1004C3007F90122531500302065D7FAA12272C90DC
:1004D30080E2E0FB7D017F90122531500302065D2F
:1004E300C20F1226FA9080E2E025E024BFF582E4F1
:1004F3003480F583EFF0D20F1226FA9080E2E0FE0B
:1005030025E024C0F582E43480F583EFF074232ED4
:10051300F582E43481F5837401F02007030205DCDE
:10052300C207300968EE25E024BFF582E43480F584
:1005330083E0753C00F53D30E70BE4253DF53D7464
:10054300FF353CF53CE53D25E0F53DE53C33F53C29
:100553009080E2E025E024C0F582E43480F583E076
:100563006003433D019080E97448F0A37461F0E4B3
:10057300A3F09080E2E024809080ECF0A37402F07A
:10058300A3E53DF0E53CA3F0753B0780399080E996
:100593007404F0A37421F09080E2E09080EBF025E6
:1005A300E024C0F582E43480F583E09080ECF090A1
:1005B30080E2E025E024BFF582E43480F583E09017
:1005C30080EDF0753B057B017A8079E9A209920FF2
:1005D300C210AD3B1223CFD2079080E2E0FF245339
:1005E300F582E43480F583E4F0EF25E024BFF5825F
:1005F300E43480F583E0FFF53B533B80E53B6055F6
:100603009080E2E0FE25E024BFF582E43480F583A8
:10061300EFF4F074532EF582E43480F5837402F022
:100623009080E2E0FF25E024C0F582E43480F58386
:10063300E05480F0EF25E024C0F582E43480F583B4
:10064300E070129080E2E025E024BFF582E434807C
:0D065300F583E004F01228DF800312260278
:0306600030036AFA
:10066300C2031220C6300762C20730092A9080E90C
:100673007448F0A37461F0E4A3F0A37488F0A37446
:1006830002F09080F9E09080EEF09080F8E09080A6
:10069300EFF0753B0780209080E97405F0A3742088
:1006A300F0A3E58BF0A3E58DF0908101E09080ED60
:1006B300F0E4A3F0753B067B017A8079E9A2099205
:0A06C3000FC210AD3B1223CFD20787
:1006CD002018030213443091030208939080E3E055
:1006DD009080D4F0E4A3F0C200E47811F620900BE2
:1006ED009080D4E004F0D2003090FD20920B9080E9
:1006FD00D4E014F0D2003092FD201803020874E407
:10070D00F524AF240524745B2FF582E43480F58342
:10071D007402F0AF240524745B2FF582E43480F568
:10072D0083E4F0AF240524745B2FF582E43480F567
:10073D00837401F0AF240524745B2FF582E43480BB
:10074D00F583740FF09080D5E0FFD20FD2101228F0
:10075D0026AE240524745B2EF582E43480F583EFF8
:10076D00F09080D4E0FF12293DD20FD2101228262E
:10077D00AE240524745B2EF582E43480F583EFF00E
:10078D009080D4E0FF12293DC20FC210122826AE70
:10079D00240524745B2EF582E43480F583EFF07428
:1007AD005B2524F582E43480F583E05480F0AF249A
:1007BD000524745B2FF582E43480F583C083C082F9
:1007CD00E0FB9080D5E0FFC20FC210122826EB4F40
:1007DD00D082D083F0E4F538753901745B2539F595
:1007ED0082E43480F583E02538F5380539E539B4F0
:1007FD0008E96338FFE53824FD600824FA60042415
:10080D00077011AF240524745B2FF582E43480F555
:10081D00837409F0AF240524745B2FF582E43480D2
:10082D00F583E538F0AF240524745B2FF582E434AD
:10083D0080F5837403F0AF240524745B2FF582E4F7
:10084D003480F583E4F0AF240524745B2FF582E446
:10085D003480F583E4F090810FF0D20A908122E587
:10086D0024F0C2183018FD2091030206E6D20C3098
:10087D0000149080D4E0540F9080E3F09080DBF072
:10088D00F4A3F012298A309003020A0DD20CC20093
:10089D00E47811F620910AA209B39209D2003091A1
:1008AD00FD20920AA209B39209D2003092FD2018C0
:1008BD00030209F4E4F524AF240524745B2FF582BB
:1008CD00E43480F5837402F0AF240524745B2FF5B6
:1008DD0082E43480F583E4F0AF240524745B2FF5B6
:1008ED0082E43480F5837401F0AF240524745B2F0A
:1008FD00F582E43480F583740FF0AF240524745B26
:10090D002FF582E43480F583E4F03009047F7A809A
:10091D00027FCEAE240524745B2EF582E43480F57F
:10092D0083EFF03009047F7380027F76AE240524B7
:10093D00745B2EF582E43480F583EFF03009047F8B
:10094D003E80027F06AE240524745B2EF582E434CE
:10095D0080F583EFF0E4F538753901745B2539F5D1
:10096D0082E43480F583E02538F5380539E539B46E
:10097D0008E96338FFE53824FD600824FA60042493
:10098D00077011AF240524745B2FF582E43480F5D4
:10099D00837409F0AF240524745B2FF582E4348051
:1009AD00F583E538F0AF240524745B2FF582E4342C
:1009BD0080F5837403F0AF240524745B2FF582E476
:1009CD003480F583E4F0AF240524745B2FF582E4C5
:1009DD003480F583E4F090810FF0D20A908122E506
:1009ED0024F0C2183018FD20900302089DD20C305F
:1009FD00000E3009047F0080027F018F241229A18F
:100A0D00309203020B909080E8E09080D4F0E4A344
:100A1D00F0C200E47811F62090139080E8E004F025
:100A2D00E0D394084002E4F0D2003090FD20911400
:100A3D009080E8E014F0E0C3940050037408F0D205
:100A4D00003091FD201803020B7DE4F524AF240541
:100A5D0024745B2FF582E43480F5837402F0AF24A7
:100A6D000524745B2FF582E43480F583E4F0AF2424
:100A7D000524745B2FF582E43480F5837401F0AFA7
:100A8D00240524745B2FF582E43480F583740FF014
:100A9D00AF240524745B2FF582E43480F583E4F0F4
:100AAD00AF240524745B2FF582E43480F583E4F0E4
:100ABD009080E8E0FF12293DC20FC210122826AE29
:100ACD00240524745B2EF582E43480F583EFF0AFBA
:100ADD00240524745B2FF582E43480F583E4F0F56E
:100AED0038753901745B2539F582E43480F583E07E
:100AFD002538F5380539E539B408E96338FFE538A7
:100B0D0024FD600824FA600424077011AF24052425
:100B1D00745B2FF582E43480F5837409F0AF2405FE
:100B2D0024745B2FF582E43480F583E538F0AF242F
:100B3D000524745B2FF582E43480F5837403F0AFE4
:100B4D00240524745B2FF582E43480F583E4F0AF43
:100B5D00240524745B2FF582E43480F583E4F09052
:100B6D00810FF0D20A908122E524F0C2183018FDD1
:100B7D00209203020A20D20C3000089080E8E0FF9A
:100B8D001229ABE4F524AF240524745B2FF582E420
:100B9D003480F5837402F0AF240524745B2FF58245
:100BAD00E43480F583E4F0AF240524745B2FF582E3
:100BBD00E43480F5837401F0AF240524745B2FF5C4
:100BCD0082E43480F583740FF09080D5E0FFC394F8
:100BDD001050067E007F008007D20FD210122826FB
:100BED00AE240524745B2EF582E43480F583EFF09A
:100BFD009080D4E0FFD20FD210122826AE24052407
:100C0D00745B2EF582E43480F583EFF09080D4E0B0
:100C1D00FFC20FC210122826AE240524745B2EF5D8
:100C2D0082E43480F583EFF0745B2524F582E4349F
:100C3D0080F583E05480F0745B2524F582E43480E4
:100C4D00F583C083C082E0FB9080D5E0FFC20FC268
:100C5D0010122826EB4FD082D083F0AF24052474D8
:100C6D005B2FF582E43480F583E06480F0E4F538A1
:100C7D00753901745B2539F582E43480F583E025FF
:100C8D0038F5380539E539B408E96338FFE5382416
:100C9D00FD600824FA600424077011AF2405247444
:100CAD005B2FF582E43480F5837409F0AF240524BD
:100CBD00745B2FF582E43480F583E538F0AF2405BD
:100CCD0024745B2FF582E43480F5837403F0AF2434
:100CDD000524745B2FF582E43480F583E4F0AF24B2
:100CED000524745B2FF582E43480F583E4F0AF24A2
:100CFD000524745B2FF582E43480F5837402F0854E
:100D0D002439AF240524745B2FF582E43480F583F8
:100D1D00E4F0AF240524745B2FF582E43480F58371
:100D2D00E4F0AF240524745B2FF582E43480F58361
:100D3D00740FF09080D7E0FFD20FD210122826AE9C
:100D4D00240524745B2EF582E43480F583EFF09056
:100D5D0080D8E0FFD20FD210122826AE24052474BD
:100D6D005B2EF582E43480F583EFF09080D8E0FFC0
:100D7D00C20FC210122826AE240524745B2EF582F4
:100D8D00E43480F583EFF09080D7E0FFC20FC210FE
:100D9D00122826EF4480FFAE240524745B2EF582C5
:100DAD00E43480F583EFF0E4F538E539C39524504C
:100DBD0014745B2539F582E43480F583E02538F52C
:100DCD0038053980E56338FFE53824FD600824FADD
:100DDD00600424077011AF240524745B2FF582E4A1
:100DED003480F5837409F0AF240524745B2FF582EC
:100DFD00E43480F583E538F0AF240524745B2FF5DA
:100E0D0082E43480F5837403F0AF240524745B2FE2
:100E1D00F582E43480F583E4F0AF240524745B2F70
:100E2D00F582E43480F583E4F0AF240524745B2F60
:100E3D00F582E43480F5837402F0E4F539AF2405CE
:100E4D0024745B2FF582E43480F583E4F0AF240540
:100E5D0024745B2FF582E43480F5837409F0AF249C
:100E6D000524745B2FF582E43480F5837403F0253B
:100E7D0039F539AF240524745B2FF582E43480F500
:100E8D0083740FF02539F539908031E06043AF243C
:100E9D000524745B2FF582E43480F583E4F0AF24F0
:100EAD000524745B2FF582E43480F583E4F0AF24E0
:100EBD000524745B2FF582E43480F583E4F0AF24D0
:100ECD000524745B2FF582E43480F583E4F0020F82
:100EDD00B1908053E0B40211AF240524745B2FF55B
:100EED0082E43480F5837409F0908053E0FFAE24E2
:100EFD000524745B2EF582E43480F583EFF0EF2545
:100F0D0039F5399080BFE0FF12293DC20FD2101282
:100F1D002826EF4401FF745B2524F582E43480F527
:100F2D0083EFF0745B2524F582E43480F583E025AE
:100F3D0039F53905249080C0E07017AF240524746D
:100F4D005B2FF582E43480F583743FF02539F53954
:100F5D008015AF240524745B2FF582E43480F5836E
:100F6D00746DF02539F5399080BFE0FF12293DD21F
:100F7D000FC2101228268F38E538B43F12AF240562
:100F8D0024745B2FF582E43480F583E4F08015AF93
:100F9D00240524745B2FF582E43480F583E538F065
:100FAD002539F5396339FFE53924FD600824FA60E8
:100FBD000424077011AF240524745B2FF582E434EB
:100FCD0080F5837409F0AF240524745B2FF582E45A
:100FDD003480F583E539F0AF240524745B2FF58259
:100FED00E43480F5837403F0AF240524745B2FF58E
:100FFD0082E43480F583E4F0AF240524745B2FF58F
:10100D0082E43480F583E4F0AF240524745B2FF57E
:10101D0082E43480F5837402F0E4F539AF240524BD
:10102D00745B2FF582E43480F583E4F0AF2405245E
:10103D00745B2FF582E43480F5837409F0AF2405D9
:10104D0024745B2FF582E43480F5837402F0053946
:10105D000539AF240524745B2FF582E43480F583C4
:10106D00740FF02539F539908032E06043AF2405D7
:10107D0024745B2FF582E43480F583E4F0AF24050E
:10108D0024745B2FF582E43480F583E4F0AF2405FE
:10109D0024745B2FF582E43480F583E4F0AF2405EE
:1010AD0024745B2FF582E43480F583E4F002119013
:1010BD00908054E0B40211AF240524745B2FF582A7
:1010CD00E43480F5837409F0908054E0FFAE24057C
:1010DD0024745B2EF582E43480F583EFF0EF25392F
:1010ED00F5399080C1E0FF12293DC20FD2101228B0
:1010FD0026EF4401FF745B2524F582E43480F583EB
:10110D00EFF0745B2524F582E43480F583E0253916
:10111D00F53905249080C2E07017AF240524745B67
:10112D002FF582E43480F583743FF02539F539804D
:10113D0015AF240524745B2FF582E43480F5837498
:10114D006DF02539F5399080C1E0FF12293DD20FA0
:10115D00C2101228268F38E538B43F12AF2405246B
:10116D00745B2FF582E43480F583E4F08015AF24B1
:10117D000524745B2FF582E43480F583E538F02582
:10118D0039F5396339FFE53924FD600824FA600427
:10119D0024077011AF240524745B2FF582E434808D
:1011AD00F5837409F0AF240524745B2FF582E434C4
:1011BD0080F583E539F0AF240524745B2FF582E4C7
:1011CD003480F5837403F0AF240524745B2FF5820E
:1011DD00E43480F583E4F0AF240524745B2FF582AD
:1011ED00E43480F583E4F0AF240524745B2FF5829D
:1011FD00E43480F5837402F0852439AF240524741A
:10120D005B2FF582E43480F583E4F0AF240524747C
:10121D005B2FF582E43480F5837404F0AF2405244C
:10122D00745B2FF582E43480F583740FF09080FFAA
:10123D00E0FF12293DD20FD210122826AE2405242C
:10124D00745B2EF582E43480F583EFF0908102E03B
:10125D00FF12293DD20FD210122826AE2405247478
:10126D005B2EF582E43480F583EFF0908102E0FF90
:10127D0012293DC20FC210122826AE240524745B1C
:10128D002EF582E43480F583EFF09080FFE0FF12BD
:10129D00293DC20FC210122826EF4480FFAE24054F
:1012AD0024745B2EF582E43480F583EFF0E4F53899
:1012BD00E539C395245014745B2539F582E43480E7
:1012CD00F583E02538F538053980E56338FFE538D5
:1012DD0024FD600824FA600424077011AF2405244E
:1012ED00745B2FF582E43480F5837409F0AF240527
:1012FD0024745B2FF582E43480F583E538F0AF2458
:10130D000524745B2FF582E43480F5837403F0AF0C
:10131D00240524745B2FF582E43480F583E4F0AF6B
:10132D00240524745B2FF582E43480F583E4F0C248
:10133D0018908122E524F02014030200BD30A8038B
:10134D000200BDC214E4F536F5377524029081C252
:10135D00E0FF24FEFEE524C39E501874C32524F53A
:10136D0082E43481F583E02536F5362537F53705EA
:10137D002480DA74C12FF582E43481F583E065367B
:10138D0060030200BD9081C2E024C2F582E4348185
:10139D00F583E0653760030200BD9081DCE06407F2
:1013AD006005C2050200BDD2059081DBE075F00A33
:1013BD0084E5F060030200BD9081D8E0FF12293D65
:1013CD00908116EFF09081D7E0FF12293D908117A3
:1013DD00EFF09081D6E09081D5E024002430FF120B
:1013ED00293D908118EFF09081DBE0FF12293D90AF
:1013FD008112EFF09081DAE0FF12293D908113EF19
:10140D00F09081D9E0FF12293D908114EFF0C2AC2C
:10141D0012275AD20CD2AC2009030214F09081D9B4
:10142D00E0F52B9081D8E0F5289081D7E0F5279055
:10143D0081D6E0FE9081D5E07C002400F526EC3EBF
:10144D00F5259081DAE0F52AA3E0F529752C0075D4
:10145D002D00752E25752F00753000753129852FBE
:10146D0041853042853143AB2CAA2DA92E1222B6CF
:10147D008F358E348D338C32AF35AE34AD33AC32D7
:10148D00E47B01FAF9F81219D78F358E348D338C30
:10149D00329080437401F0A37418F0A37480F0A30C
:1014AD007401F0A37406F0A3E535F0A3E534F0A3C1
:1014BD00E533F0A3E532F0E4A3F0A3F09081C2741C
:1014CD000BF0200703021644C2077A807943E0FD32
:1014DD00A209920FD2101223CF4003021644D20656
:1014ED00021644908114E0FD54F0FEC4540F2430D4
:1014FD00908011F0ED540F2430A3F0908113E0FD96
:10150D0054F0FEC4540F2430908013F0ED540F248A
:10151D0030A3F0908112E004F0E0FD54F0FEC454CD
:10152D000F2430908015F0ED540F2430A3F09080EF
:10153D00187441F0908116E0FD54F0FEC4540F2450
:10154D0030908020F0ED540F2430A3F0908117E0FF
:10155D00FD54F0FEC4540F2430908022F0ED540F52
:10156D002430A3F0908118E0FD54F0FEC4540F24F4
:10157D0030908024F0ED540F2430A3F0752401E455
:10158D00F53974092524F582E43480F583E0642A65
:10159D00601274C32524F582E43481F583E0623949
:1015AD00052480DE0524E53954F0FFC4540FF538C9
:1015BD00D394095014E5382430FF74092524F5829D
:1015CD00E43480F583EFF08012E5382437FF740999
:1015DD002524F582E43480F583EFF00524E53954B4
:1015ED000FF538D394095014E5382430FF740925CC
:1015FD0024F582E43480F583EFF08012E53824374A
:10160D00FF74092524F582E43480F583EFF0908191
:10161D00C27428F0300720C207E0FD14908009F055
:10162D00A37424F07B017A807909A209920FD2105C
:10163D001223CF5002D206300607C206D20702008F
:0B164D00BDC289D2A89081047416F081
:031658000200BDD0
:01165B00226C
:0A299600E4FEEEC39F50030E80F82C
:0129A0002214
:0D297000904001E04440F07F1412299622AF
:0D297D00904001E054BFF07F141229962213
:0F295100122970C210309502D21012297DA210E7
:012960002254
:02272C00AD07F7
:10272E00E4FCED30E709904001E04420F080079092
:10273E004001E054DFF0122951ED25E0FD0CBC08FC
:0B274E00E1904001E04420F01229510E
:01275900225D
:1026FA00E4FDFC12295150010DED25E0FD0CBC074B
:10270A00F212295150010D904001E054DFF0300FD0
:10271A0004E04420F0122951904001E04420F0AF37
:01272A0005A9
:01272B00228B
:02253100AC07F5
:10253300EB6009904001E04480F08007904001E0A7
:10254300547FF012297D904001E04420F07F141263
:102553002996122970904001E054DFF07F1412296C
:102563009612297DE4FFEB600514FE25E0FFEC2DB8
:052573002FFF12272CD0
:012578002240
:1028DF0012297D904001E054DFF07F1412299612E7
:0A28EF002970904001E04420F0221F
:0F29610045746865726E6574206661696C21004B
:10248200602C8229FFFFFFFFFFFFFFFFFFFFFFFF1F
:10249200FACE000000000000000000000000000072
:1024A200000000000000000000000000000000002A
:1024B2005E825C08004500002D007B400040113A1E
:1024C2004600000000FFFFFFFF03CD03CD0019000F
:0124D2000009
:101FFE00D2B47F64122996C2B47F641229969003DC
:10200E00007421F07811E62402FF7811E6B507027C
:10201E00D322900300E0B421F190030E7448F090A7
:10202E00030AE4F0A3F0A3F0A37402F0900301748A
:10203E0044F0A3744FF0A37444F090030774FFF0C0
:10204E0090030F7401F0900308E4F0A3F0A3742042
:10205E00F0A3E4F0900300740AF0754A01754B8208
:10206E00754C2FE4FE900310E0FD784AE475F00104
:10207E00121A57ED12186E900310E0FF0EBE06E511
:10208E009003007461F0754A01754B82754C2FE414
:10209E00FE784AE475F001121A57121828900301BF
:1020AE00F00EBE06EC9003077444F0900300742209
:0720BE00F090030DE4F0C3F4
:0120C50022F8
:1027B10090030AE4F0A3F09003007422F090030860
:1027C100E4F0A37440F0EF2410FFA3F0A3E4F09031
:0827D10003007422F07412F001
:0127D90022DD
:062869008B488A49894AF0
:10286F00E4FFEFC39D50137848E475F001121A5737
:0A287F00121828900310F00F80E8F3
:01288900222C
:102802007548037549E8301312E5491549700215F8
:10281200481445487005121FFED322900300E020A1
:03282200E2E4C32A
:012825002290
:101F2C008B448A4589468D47A2129213122802507F
:101F3C00012290030AE4F0A3F09003007422F090C5
:101F4C000308E4F0A37440F0E547D394404007E560
:101F5C00472410FF80027F4090030AEFF0A3E4F0C7
:101F6C009003007422F07412F07B017A8279297D3F
:101F7C00061228697B017A82792F12286920111E9A
:101F8C0090823574FAF0A374CEF0A3E547F0E4A385
:101F9C00F07B017A8279357D04122869801EE54731
:101FAC00240E908277F07B017A82795C7D1E122858
:101FBC00697B017A82792F7D06122869AB44AA4588
:101FCC00A946AD471228699003047440F0E547D345
:101FDC0094404008E5472410A3F080069003057454
:101FEC0040F0900306E4F02012069003007426F0F3
:021FFC00C322FE
:062229008B448A45894642
:10222F00ED2404FF7E04EEC39F501C7844E475F048
:10223F0001121A57121828FD742B2EF582E43481DF
:10224F00F583EDF00E80DFE4FDFCFEEF30E0107B58
:10225F00000EEB242BF582E43481F583E0FD1FEEB5
:10226F00C39F5022AB060E742B2BF582E43481F5FD
:10227F0083E06204AB060E742B2BF582E43481F5F8
:10228F0083E0620580D9AF060E742B2FF582E434FC
:10229F0081F583ECF0AF060E742B2FF582E43481B9
:0622AF00F583EDF0AF061F
:0122B5002206
:0823CF008B3F8A4089418D42D9
:1023D700200F1A90812B74FFF0A3F0E4A3F0A374ED
:1023E7001FF0122229E5422406F543802BE4F5432A
:1023F700E543C39542501E783FE475F001121A5722
:10240700121828FF742B2543F582E43481F583EFF6
:10241700F0054380DB8542437B017A81792BA20F4C
:102427009211A2109212AD43121F2C501C7BFF7AFF
:102437002979617D0F122229AD077BFF7A297961FE
:0A244700C211C212121F2CD322C3CF
:012451002268
:0729B5009003007426F022DC
:10257900C292D292E47811F6758911758815D28DB7
:10258900438E0275C83C75CDFF75CBFF75CCD975E7
:10259900CAD9C204759850D2AFD2A9D2ACC297C2D7
:1025A90096D218C21690822704F012297D780076F7
:0525B900FF1229702251
:0300130002288A36
:10288A00C0E0C083C082908103E014F0E07006C209
:0E289A008EC2AAD203C28BD082D083D0E0328D
:1026C6000000001F003B005A0078009700B500D4B8
:1026D60000F301110130014E016D0000001F003CA6
:1026E600005B0079009800B600D500F401120131B4
:0426F600014F016E21
:062186008B5F8A60896195
:10218C00121955AEF0244EF563EE34F8F56290005A
:10219C000212184124FFF565E434FFF564E563246D
:1021AC0001FFE43562FE7C007D04121909AA06AB1E
:1021BC0007AE62AF637C017D6D1218A2EF2BFDEEB2
:1021CC003AFCE56525E0FFE56433FE74C62FF58225
:1021DC0074263EF5837401932DFFE4933CFEAB5FB4
:1021EC00AA609000031218417C002FFFEC3ECF2414
:1021FC00FFCF34FFAB07FAAE62AF637D041219094F
:10220C00ED64024C7012C3E5659402E5646480943D
:0C221C008040050BBB00010AAE02AF03BE
:012228002293
:0A1B35008E5F8F608B618A62896306
:101B3F00EE3395E08F6D8E6CF56BF56AE47F04FEE6
:101B4F00FDFCAB6DAA6CA96BA86A1219E4EF240215
:101B5F00FFE43EFEE43DFDE43CFCE47BB57A05F991
:101B6F00F81225BE8E648F65E5652401FFE43564A8
:101B7F00FE7C007D04121909AA06AB07AE64AF659F
:101B8F007C017D6D1218A2EF2BFFEE3AFEC3E560CC
:101B9F009FF569E55F9EF568AE64AF651C7D041225
:101BAF001909ED64024C70087BFF7A2679E08006F4
:101BBF007BFF7A2679C67D017C00ED25E0FFEC33B3
:101BCF008F82F583121980FFC3E5699FE5F064806A
:101BDF00F8E568648098400B0DBD00010CED640CB6
:101BEF004C70D7ED24FFFFEC34FFFEEF25E0FFEE46
:101BFF00338F82F583121980FFAEF0C3E5699FF52D
:101C0F0067E5689EF566E56524B2FFE5643407ABCA
:101C1F0061AA62A9638FF01219B8AB61AA62A963B6
:101C2F00900002ED121880E56704900003121880EF
:011C3F002282
:10291200EF2403FFE43EFE7C007D07121909ED243B
:0629220001FFE43CFE226F
:081D43008F4E8E4D8D4C8C4B30
:101D4B007B807A51790178001225BE8E4F8F507BA4
:101D5B00007A007953121B3575550375561F7B009E
:101D6B007A0079531221868E4F8F501229127C00E4
:101D7B007D071219098C518D52C3E5509552FFE521
:101D8B004F9551FE3395E0FDFC7B807A51790178BC
:101D9B00001219E4EF2420F55AEE341CF559E43DFA
:101DAB00F558E43CF55775550A75561F7B007A00BC
:101DBB0079531221868E4F8F501229127C007D078A
:101DCB001219098C518D52C3E5509552FFE54F9571
:101DDB0051FE3395E0FDFC7B807A5179017800123E
:101DEB0019E4EF2420F55EEE341CF55DE43DF55C63
:101DFB00E43CF55BAF5AAE59AD58AC57AB4EAA4D60
:101E0B00A94CA84BC3121A415004E4FEFF22AF5E4B
:101E1B00AE5DAD5CAC5BAB4EAA4DA94CA84BC312EF
:0C1E2B001A414004E4FEFF227E007F010B
:011E37002288
:0E1C40008F418E408D3F8C3E8B428A438944FB
:101C4E00908110E0FEA3E0FFE4FCFDE5412FF5419D
:101C5E00E5403EF540ED353FF53FEC353EF53EE5D2
:101C6E00486025AF41AE40AD3FAC3E121D43EF4E36
:101C7E006016E5412410F541E540340EF540E4359B
:101C8E003FF53FE4353EF53EE54445434542601C95
:101C9E007B807A5179017800AF41AE40AD3FAC3ECA
:101CAE001225BEAB42AA43A944121B35E547454651
:101CBE0045457003021D42AF41AE40AD3FAC3E7B89
:101CCE00807A51790178001225BEAC00AD01AE02CA
:101CDE00AF038F418E408D3F8C3EE47B107A0EF920
:101CEE00F81225BEAB45AA46A947900002EF12187E
:101CFE0080E47B107A0EF9F8AF41AE40AD3FAC3EBA
:101D0E001225BEAE02AF038E498F4A7C007D3C1277
:101D1E001909AB45AA46A947900001EF121880AEEB
:101D2E0049AF4A7C007D3C121909AB45AA46A9472A
:041D3E00ED12186E1C
:011D4200227E
:1022B600122186EE3395E0FDFC7B807A5179017818
:1022C600001219E4C004C005C006C007AB41AA420B
:1022D600A943900002121841FFE4FCFDFE7B107A30
:1022E6000EF9F81219E4D003D002D001D000121969
:1022F600D7C004C005C006C007AB41AA42A9439097
:102306000001121841FFE4FCFDFE7B3CFAF9F812CD
:1023160019E4D003D002D001D0001219D7A804C006
:1023260005C006C007AB41AA42A943121828FFE41C
:0C233600FCFDFED003D002D0011219D72C
:012342002278
:03000B0002264585
:10264500C0E0C083C082C0D075D008C28D758AAF86
:10265500758C3CD2B590810FE004F0E0640A60030C
:10266500300A0AC20A201905201802D299D2027826
:102675001106E67002F5A8C2B5D0D0D082D083D0BD
:02268500E03241
:03001B000227DADF
:1027DA00C0E0C0F0C083C082C0D075D000C000C2C3
:1027EA008F908100E475F00112193FD000D0D0D04B
:0827FA0082D083D0F0D0E03260
:03002300021E3882
:0B1E3800C0E0C083C082C0D075D0188D
:101E4300209803021EE5C298301403021F233016A4
:101E53002D9081C2E024C3F582E43481F583E599B2
:101E6300F09081C2E004F09081C1E0FFA3E0C39F42
:101E73005003021F23C216C297D214021F23301726
:101E83004C9081C2E024C3F582E43481F583E59963
:101E9300F09081C2E004F0E0FFC394075003021FF7
:101EA30023C2179081C4E0646270759081C5E064B9
:101EB30001706D9081C6E064217065D2169081C770
:101EC300E02F547F9081C1F0E004F08053E599B492
:101ED300B510D2979081C3E599F09081C27401F057
:101EE300D21730993BC2993019230510908122E013
:101EF300FFE510C39F5010745B2510F582E4348016
:101F0300F583E0F5998019C219D2188013D2197597
:101F13001000745B2510F582E43480F583E0F599B5
:091F2300D0D0D082D083D0E0328E
:030003000226874B
:10268700C0E0C0F0C083C082C0D075D000C000C019
:1026970001C002C003C004C005C006C0071229B5A7
:1026A700D207C2A8D007D006D005D004D003D002E5
:0F26B700D001D000D0D0D082D083D0F0D0E0328C
:10292800438E2075D2028F828E83E0FFE4F5D25366
:042938008EDFD2AFAD
:01293C002278
:1028F900E5D220E0FBC2AF43D2028F828E83EDF096
:0929090075D25075D2A0D2AF22A4
:10165C0002181DEC5D046005E859047003021813B0
:10166C001217DE580460F6EC4860F2EC7004FDFED4
:10167C00FF22C860DB2481C85009C3986002500661
:10168C0002181A9850CAF582E9294B4A7005AB82A8
:10169C0002180975F0007C1A7880C3EF9BEE9AED66
:1016AC0099400DC3EF9BFFEE9AFEED99FDE842F0D9
:1016BC00DC23ACF0D0E0FFD0E0FED0E0FDAB82202C
:1016CC00E7101BEB60BAEC2CFCEF33FFEE33FEEDB6
:1016DC0033FD0217F5E803F830E705C0F075F000AC
:1016EC00EF2FFFEE33FEED33FD40B830E7C280AA9A
:1016FC0074F8CC6480CCC86480C8F582046043C3A1
:10170C00EB9FF5F0EA9E42F0E99D42F0E89C45F033
:10171C0060305018E5825FFFE582F42B5582FB5058
:10172C00210ABA001D09B90019088016E5825BFB75
:10173C00E582F42F5582FF50090EBE00050DBD0049
:10174C00010CC3EB9FF5F0EA9E42F0E99D42F0E8F4
:0D175C009C45F06007CC4820E701B3EC226B
:1017690075F020800E75F010800575F0087D007EFB
:10177900007F003392D530D503121A33EC33401071
:10178900EF33FFEE33FEED33FDEC33FCD5F0ED2204
:0E179900E5F0247EA2D513CC92E7CDCEFF2240
:1017A700EDD2E7CD33EC3392D524814006E4FFFE3A
:1017B700FDFC22FCE4CFCECDCC24E0501174FF8099
:1017C700EDC3CC13CCCD13CDCE13CECF13CF047036
:0717D700F030D5DE021A33E9
:1017DE00E9D2E7C933E833F892D5EDD2E7CD33EC51
:0717EE0033FC5002B2D522CA
:1017F500EC30E7100FBF000C0EBE00080DBD000455
:101805000BEB6014A2D5EB13FCED92E7FD2274FF00
:10181500FCFDFEFF22E480F8A2D574FF13FC7D8059
:03182500E480EF6D
:10234F00020026E493A3F8E493A34003F68001F27E
:10235F0008DFF48029E493A3F85407240CC8C3338F
:10236F00C4540F4420C8834004F456800146F6DF5E
:10237F00E4800B0102040810204080902452E47E78
:10238F00019360BCA3FF543F30E509541FFEE49353
:10239F00A360010ECF54C025E060A840B8E493A31A
:1023AF00FAE493A3F8E493A3C8C582C8CAC583CA45
:1023BF00F0A3C8C582C8CAC583CADFE9DEE780BEFD
:0124D3000008
:10182800BB010689828A83E0225002E722BBFE02BE
:09183800E32289828A83E49322F1
:10184100BB010CE58229F582E5833AF583E022505C
:1018510006E92582F8E622BBFE06E92582F8E222A6
:0D186100E58229F582E5833AF583E49322C0
:10186E00BB010689828A83F0225002F722BBFE0159
:02187E00F32253
:10188000F8BB010DE58229F582E5833AF583E8F09E
:10189000225006E92582C8F622BBFE05E92582C84A
:0218A000F22232
:1018A200EF8DF0A4A8F0CF8CF0A428CE8DF0A42E5A
:0218B200FE2214
:1018B400BC000BBE0029EF8DF084FFADF022E4CC18
:1018C400F875F008EF2FFFEE33FEEC33FCEE9DECE1
:1018D400984005FCEE9DFE0FD5F0E9E4CEFD22ED27
:1018E400F8F5F0EE8420D21CFEADF075F008EF2F71
:1018F400FFED33FD4007985006D5F0F222C398FD62
:051904000FD5F0EA22FE
:10190900C2D5EC30E709B2D5E4C39DFDE49CFCEEF9
:1019190030E715B2D5E4C39FFFE49EFE1218B4C3A5
:10192900E49DFDE49CFC80031218B430D507C3E4A0
:061939009FFFE49EFE2268
:10193F00C5F0F8A3E028F0C5F0F8E5821582700233
:06194F001583E038F022D0
:10195500BB010A89828A83E0F5F0A3E0225006875D
:10196500F009E71922BBFE07E3F5F009E31922891F
:0B197500828A83E493F5F07401932252
:10198000BB0110E58229F582E5833AF583E0F5F0A5
:10199000A3E0225009E92582F886F008E622BBFE82
:1019A0000AE92582F8E2F5F008E222E5832AF583C8
:0819B000E993F5F0A3E993228D
:1019B800BB010A89828A83F0E5F0A3F0225006F77A
:0F19C80009A7F01922BBFE06F3E5F009F3192277
:0D19D700EF2BFFEE3AFEED39FDEC38FC225F
:1019E400E88FF0A4CC8BF0A42CFCE98EF0A42CFCA2
:1019F4008AF0EDA42CFCEA8EF0A4CDA8F08BF0A420
:101A04002DCC3825F0FDE98FF0A42CCD35F0FCEB7E
:101A14008EF0A4FEA9F0EB8FF0A4CFC5F02ECD3943
:0F1A2400FEE43CFCEAA42DCE35F0FDE43CFC22B0
:1025BE00C2D5E830E70FB2D5E4C39BFBE49AFAE448
:1025CE0099F9E498F8EC30E717B2D51225F4121AFF
:1025DE00A3E4C39BFBE49AFAE499F9E498F8800328
:1025EE00121AA330D50DE4C39FFFE49EFEE49DFDB9
:0425FE00E49CFC223B
:0E1A3300C3E49FFFE49EFEE49DFDE49CFC22C4
:101A4100EB9FF5F0EA9E42F0E99D42F0EC6480C81C
:061A510064809845F022BC
:101A5700FAE6FB0808E6F925F0F618E6CA3AF62290
:101A670075F008758200EF2FFFEE33FECD33CDCC36
:101A770033CCC58233C5829BED9AEC99E5829840B9
:101A87000CF582EE9BFEED9AFDEC99FC0FD5F0D696
:101A9700E4CEFBE4CDFAE4CCF9A88222B800C1B9C0
:101AA7000059BA002DEC8BF084CFCECDFCE5F0CBFE
:101AB700F97818EF2FFFEE33FEED33FDEC33FCEB37
:101AC70033FB10D703994004EB99FB0FD8E5E4F9F2
:101AD700FA227818EF2FFFEE33FEED33FDEC33FCDF
:101AE700C933C910D7059BE99A4007EC9BFCE99AD3
:101AF700F90FD8E0E4C9FAE4CCFB2275F010EF2F18
:101B0700FFEE33FEED33FDCC33CCC833C810D70717
:101B17009BEC9AE899400AED9BFDEC9AFCE899F852
:0E1B27000FD5F0DAE4CDFBE4CCFAE4C8F922E5
:00000001FF
